:10740000E0E0F0E0859194910196089520E82093C2
:1074100061001092610081E085BF82E085BF80EF4E
:1074200085B987EE84B91DB8769A10BA80EF81BB12
:1074300082E68BB983EF8AB980E58CBD81E08DBD92
:10744000089580EE8BB98BEA55D0109289008AEFAF
:107450008093880082E080936F0083E080938100B6
:10746000E7E0F1E05CD0ED30E9F7AFE1B4E0EDE06A
:10747000F1E003E010E101900D921A95E1F7A059B7
:10748000BF4F0A95B9F753D081E08093D7008AE4C3
:1074900082BF1092D8001092E2001092DA0010928F
:1074A000E10080E808D019BC1EBA1092E0006ED44A
:1074B00089E05AD481E98093D8000895F201F999BE
:1074C000FECFF2BDE1BD0895F9DFF89A80B508C09E
:1074D000F5DF1FBA80BD0FB6F894FA9AF99A0FBE7D
:1074E00031962F01089590E81BD08D939A95E1F77E
:1074F000089586E008D010C083E005D08F2F10D00B
:107500008E2F0ED080E05E9A59980AC005D085E093
:10751000FADF06D080FDFDCF599A5E9808958191DB
:107520008EBD8DB5000087FFFCCF8EB50895E7EEC8
:10753000F2E090EB5C98892FF3DF80E1F1DF5C9A59
:10754000EEDF87EE8E278F77D9F79395983B91F7EB
:107550000895E5EDF1E08191908101969083829309
:10756000092E0AF400940091D30106FB5EF0009608
:10757000929111F493959083000C081620F42E98A4
:107580002F982D980895937009F42E9A913009F44C
:107590002F9A923009F42D9A0895ECECF1E097813E
:1075A0009923EAF08FB18095807F669B88601C9B51
:1075B00084609581891310C09681992381F4938109
:1075C000891306C09481992396E959F080E00AC096
:1075D00083839095892304C085839AE0968380E015
:1075E0009FEF9483828308958091D30186FF2E9A22
:1075F0002F9A2D9A22243324ECECF1E01086118688
:107600001286E7EEF1E08091CE0187FD1BC084FD7C
:1076100032C082FF0895C685CC23E1F3F894289AFE
:107620000088F785E02D68DFE0E0F0E0A7EEB1E04C
:107630005ADFA7EEB1E03ED3E058FF4FCA95B1F74D
:107640006BDFC9C18301282D6090F0017090EF01BC
:1076500046D019F48823C1F70895380188243FD013
:10766000E1F58091EE01821709F483016090F20147
:107670007090F101F4CF6090F2017090F1012FD081
:1076800081F48823C1F708959FEF85FD08C086FD2A
:1076900005C083FF0895B4DEE9F39DC191E097FB37
:1076A000890E662477248301222719D0B1F4882318
:1076B00089F38091EE0136F0881650F4821730F08D
:1076C000213003C0881520F4281710F48301282FD7
:1076D0006090F2017090F101E8CF3801822EF30141
:1076E0000BDFA7EEB1E0FFDEC7EED1E0E0E0F1E0B6
:1076F00097E009908191081621F49A95D1F70880B6
:1077000080100ACFC9E0EFDECA95E9F705DF0FDF89
:047710008827089529
:1077140041524455424F59C82F258113AF0000FFF1
:10772400FFCFCFFFFFFFFFCFCFFFFF0000FE067E9E
:107734007E06FE46565616FE0656461EFE3F61E976
:10774400E3FFE3EBE3FFE3EBE3FFE16B3F12011045
:107754000102000008412337000100020100010971
:10776400023E00020100803209040000010202010D
:107774000005240010010424020405240600010766
:107784000582030800FF09040100020A0000000743
:107794000504021000010705830210000104030917
:1077A400042203410072006400750069006E006FDA
:1077B4000020004D006900630072006F002000206B
:1077C4000020001803410072006400750069006E17
:0C77D400006F0020004C004C004300003F
:1078000011241FBE8DEF9AE09EBF8DBF04B714BE3A
:1078100088E18093600010926000409100085091D0
:1078200001086F917F91A6C00F928F939F931F9233
:107830000FB60F9211244F936F938091DA0080FF5F
:107840004CC038C00F920FB68F939F93EF93FF9366
:1078500088278093850080938400ECECF1E0978189
:10786000907261F490818917980B908309F45D9868
:1078700091818917980B918309F4289896819150EA
:1078800008F096839481915008F09483881639F417
:107890007C9B05C0B5DD19F0C10101961C01FF916B
:1078A000EF915CC080E189BD82E189BD09B400FE31
:1078B000FDCF08958091D80080FF0FC08091DA003D
:1078C0008E7F8093DA008091D90080FF04C0EADFC8
:1078D00081E08EBB02C019BC1EBA8091E10080FF1E
:1078E0000BC03CD280FF08C03CD28091D80080629F
:1078F000E2DD19BC85E08EBB8091E10084FF1AC0F7
:107900002DD284FF17C0CEDF8091D8008F7DD3DDCC
:107910008FEE2AD023D28F7E816026D28091D7012C
:10792000882331F48091E30087FD02C081E001C02B
:1079300084E08EBB8091E10083FF0CC00FD283FFF7
:1079400009C087EF11D082E08EBB1092D7010BD017
:1079500008D21CD26F914F910F901F909F918F91E1
:107960000FBE0F9018958EEF0090E1000822009254
:10797000E10008954BDDA0E0B1E0E4E1F7E7059018
:107980000D92AB3CE1F71D92BB30E9F701FD0FC052
:1079900000FF03C07C9B0BC008C003FF08C06757F3
:1079A000774729F04757574711F02ADDA1F449DD01
:1079B000222433243101882492DE789447D00AD3DC
:1079C000ECDD62DE811411F00FDEF8CFC2DDC10103
:1079D000805B964398F3F89489EB8CDD81E080938B
:1079E000E00010926F0010928100109285001092BA
:1079F000840081E085BF15BEC2DD5D9828980C9497
:107A00000000A7D107C054D102C0E1D239F0A3D100
:107A100082FFFBCF85FFF7CF8091F1000895082EFC
:107A200083E098D185FD07C08DD102C0D0D269F026
:107A300092D180FFFBCF0092F1008091D30185FBB2
:107A400026F05D9A84E68093CC01089582D182FF6E
:107A50004AC18091D30185FB26F0289A84E6809361
:107A6000CD01CFDF182F853431F48CEB94E31C016A
:107A700025DD8DE008C1843511F4C3DFFACF8C34E5
:107A8000C1F38035B1F3843721F484E4C8DF80E0AA
:107A9000FAC0813611F489E5F6C0813429F4B1DFEA
:107AA000582EAFDF482EE5CF803711F483E5EBC0C9
:107AB000833539F4C0E0D1E08991B1DFC730E1F717
:107AC000E3C0863521F481E3AADF84E3DCC0863796
:107AD00061F481E3669B8E5F1C9B8F5FA0DF8FB19B
:107AE000809582958F708F5BCEC08837A9F489DF2F
:107AF0008093D301289884FD289A5D9883FD5D9A30
:107B00002E9881FD2E9A2F9882FD2F9A2D9880FD18
:107B10002D9A87FD8824ADCF8A3649F48FE9F3DCAE
:107B2000C3E0FEDC7CDFCA95E1F7F6DCADC083374D
:107B300031F487E874DF85E972DF8EE1A4C0853611
:107B400039F4E0E8F3E7C7D0E058F040E0F791CF30
:107B5000823631F489E563DF80E061DF80E893C03D
:107B6000823419F0873609F07AC02224332449DFA1
:107B7000D82F47DFC82F45DF082F8354843008F003
:107B800081C0063411F4440C551CF20110926F00B0
:107B90001736A1F4033471F483E0AFDCC1DC3FDFBE
:107BA0002197E1F7B9DC08C0063411F4859101C0D2
:107BB0008BDC35DF2197C2F72F0149C00334A1F4D4
:107BC0008E2F8F7021F495DC80E297DC9FDC91DCB6
:107BD00082E093DC16DFA4DCCA95E1F797DC3196EE
:107BE000DA9571F72F0131C00634F1F49F01F437B3
:107BF000D8F471D019C005DF063461F4C0FB46F03B
:107C0000F43728F4182E81E087BFE89511243296C6
:107C1000082E0AC0043439F4DF01B370A951BD4FF6
:107C20008D93319601C054DC21972AF7043431F446
:107C30002F01F370FE2B49F47ADC07C0063429F4D7
:107C40002F01F901F43708F444D08DE0E8DE063462
:107C500011F45694479482E080936F0015C08237E8
:107C6000E1E049F08634E0E031F08E34E3E019F0F1
:107C7000813531F4E2E0F0E089E087BF849103C010
:107C80008B3111F08FE3CBDE83E0B1D15BD095FF78
:107C900003C009C09CD139F15ED080FFFBCF52D028
:107CA00002C095D101F157D080FFFBCF84E09FD176
:107CB0008BE749C0F437B8F40ED090E40D901D90D6
:107CC00081E087BFE89532969A95C1F71124E05874
:107CD000F04085E001C083E001D081E187BFE895F5
:107CE00007B600FCFDCF08959091DF018091E0017F
:107CF000913231F0913A61F5813251F538D087C037
:107D0000803231F534D063D1E9F08530D9F023D019
:107D100083FD18C082FFF7CF04C07EDE81936150DF
:107D200031F09091F3008091F200892BB1F7C0DF20
:107D3000611549F704C04BD129F0853019F00BD0FB
:107D400080FFF9CF8EE79091E80089238093E800C7
:107D5000089584E04CD18091E80008958091E2007C
:107D60000895FCDF8E7F80618093E20008952DD11D
:107D7000E8EDF1E067E0089582E061EC09D083E08E
:107D800061E802D084E060E842E103C080E060E0A6
:107D900042E02DD181E007D01092ED006093EC001D
:107DA0004093ED0008959091EB00892B8093EB00B8
:107DB000089560E0923039F0933041F0913099F4B9
:107DC000EDE362E110C0EFE46EE30DC0813018F422
:107DD000EDE864E008C019F4E1E962E204C0823031
:107DE00011F4E3EB68E1F1E008958091DF0188236D
:107DF0004CF402C0ECD051F0AEDF82FFFBCF58CF85
:107E0000E6D021F0A8DF80FFFBCF9CDF08954091F2
:107E1000E5015091E6014617510510F490E028C0A5
:107E2000611511F0462FFACF8DDF40E0F7CFCFD0AC
:107E300059F1853049F18FDF83FD3ACF8CDF82FD28
:107E400020C080FF15C03091F3002091F20005C0E2
:107E500081918093F10041502F5F411519F0283036
:107E60003105B0F350E02830310509F451E06ADF04
:107E70004115E9F65523D9F604C0A9D029F085307B
:107E800019F069DF82FFF9CF13CFEFEDF1E0C4DD28
:107E90008193E73EE1F728DF5EDF83FF91C08091A9
:107EA000DF019091E001913009F170F09330F1F031
:107EB000953009F444C0963009F456C0983009F45E
:107EC00060C0993059F767C0823841F78091E3016B
:107ED0008DD02091EB001092E90077D02295269565
:107EE00021702093F1001092F10052C0882311F00C
:107EF0008230A1F68F71823089F68091E10188236A
:107F0000D1F42091E301277049F22093E900809198
:107F1000EB0080FF10C0933011F480E20BC080E1D1
:107F200042DF81E0880F2A95E9F78093EA001092FA
:107F3000EA0088E038DF1092E90047D02AC08823A1
:107F400091F41091E10110680FB7F8943ED04DDF25
:107F500002DF80FFFDCF1093E300103883E009F4C7
:107F600082E08EBB0FBF2CC08058823048F58091D4
:107F7000E1019091E2011DDF603011F126D047DF71
:107F80001FC08038E9F421D08091D7018093F1009F
:107F9000D9DE2BDF15C0882399F49091E10192304E
:107FA00078F49093D70111D020DF8091D7018823F6
:107FB00021F48091E30091E087FD94E09EBBDCDE3C
:107FC000CADE83FF089580E2EEDE87EFBCCE8EB37B
:107FD00088230895FCDF69F08091E9008F93109267
:107FE000E900B9DE83FF01C050DF8F918770809375
:047FF000E900089507
:047FFC005BCEFBDC81
:040000030000740085
:00000001FF
